:020000040000FA
:100000000228090083120313A001A101A2011230EA
:10001000A0003430A1005630A200B101B201B301FA
:10002000B401B501B601B701B801A401A3012C3098
:10003000A5000130A600A701A801AC01AC148530D1
:10004000A900850186018701831606309F0038309C
:100050008500860187010C10831201309000220870
:10006000AF000430B0008C202108AF000230B00097
:100070008C2020083F39AF002C08AD002C0CAD05BA
:10008000050DAD062D1B2F170130B0008C202F2839
:1000900085196F20051A5C20A20A0F3022050A3C40
:1000A0000319532808001030A207F030A205603071
:1000B000220203195C2808003F30AC05A201A10A06
:1000C0000F3021050A3C0319662808001030A107EB
:1000D000F030A1056030210203196F2808002C1AA6
:1000E000A20A2C122C1D7B282C110830AC06AC194E
:1000F000A00AAC1DA003A101A00A0F3020050A3CF4
:1001000003198728243020020319A00108001030A9
:10011000A007F030A00508002908A7070318A80ABF
:100120008030A7070318A80A0C30A8072808AD00DC
:100130000E082702031CAD030F08AD02AD1F962861
:10014000F83085052F08860030088504FF30851EAD
:1001500000302C060139031DBB20A30A0319A40A91
:1001600026082402031D080025082302031D080099
:100170007021482008002B082402AE002A08230220
:10018000031CAE03AD002C1CDC282C102E08031D14
:1001900005292D084B3C031C05290A302D02031CA0
:1001A000052928302D02B10CB20CB30CB40CB50CDF
:1001B000B60CB70CB80C08002C142E080319F12843
:1001C000023C031C0529AE1CF128AC1C0B21B1011B
:1001D000B201B301B401B501B601B701B801B1175D
:1001E000AC1024082602AE0023082502031CAE032F
:1001F000AD002E08031D02292D08963C031C022980
:10020000AC1C4820AC1C70210629AC142308AA00A1
:100210002408AB000800103038063F39031D0800E1
:10022000B51C08002C11B61A2C15C0303605403A02
:100230000319AC15C03A0319AC112C1235182C1641
:10024000340CAE00350CAD00AE0CAD0C2D08AE007C
:10025000AE0CAE062E08AE0CAE0CAE062E08AE0CE2
:10026000AE0CAE0CAE0CAE062E1846292D080F397A
:10027000093C031C46292D087039503C031C4629B3
:100280002D087F39A100A20170212C17330C340CEA
:10029000AD002D0C7F39AD00AE00AE00AE0CAE0649
:1002A0002E08AE0CAE0CAE062E08AE0CAE0CAE0C8C
:1002B000AE0CAE062E186F292D080F39093C031C11
:1002C0006F292D083039203C031C6F292D083F3938
:1002D000233C031C6F292D083F39A000AC170800F0
:1002E00001302407A6002C3023070318A60AA50016
:0202F000080004
:02400E00393B3C
:00000001FF
